:10000000ADC0189501C018950FB617EE12BF7395C5
:1000100080FF0BC00894809B88944795783019F432
:10002000112719BF82600FBE1895713011F4919895
:10003000FACF7A3029F4919A112719BF8160F3CF52
:1000400040FD919A40FF91984695EDCF81E012E0F6
:1000500013BF899A889808958827772712E019BFD7
:1000600080FFFECF0895809BFECF8099FECF1BEDD1
:1000700012BF12E018BF19BF772781FFFECF8D7F17
:1000800008952FEF2A95F1F71A95D9F7089518E0FA
:10009000331F10F4C69A01C0C698C79A26E02A9565
:1000A000F1F7C79821E02A95F1F71A9589F7089595
:1000B00018E030E0330FB5993160C79A26E02A95F1
:1000C000F1F7C79821E02A95F1F71A9599F7089565
:1000D00000001FED17BBC798063829F0C49A1FEF20
:1000E000D0DFC49804C0C4981FEFCBDFC49A1FEFC1
:1000F000C8DF3CEACCDF33E5CADF0032B8F00023CA
:10010000AAF0A0E2D5DF333599F030E0C0DFC79A1E
:1001100026E02A95F1F7C79821E02A95F1F73CEA05
:10012000B6DF33E5B4DFAA9569F702C030E0AFDF90
:10013000063811F030E0ABDF10E1A3DF089541E4B1
:100140008BDF46E589DF42E587DF40E285DF49E472
:1001500083DF43E581DF40E57FDF089511271BBF83
:100160001FEF12BBC49A18BB10E117BB6FDF789466
:100170007ADF4B31E9F3443519F475DF042F3CC1C4
:10018000433511F4DCDFF4CF463529F442E364DF74
:1001900040E362DFEDCF463729F441E35DDF40E322
:1001A0005BDFE6CF443799F442E156DF43E154DFA9
:1001B00040E252DF48E250DF48E34EDF48E44CDFE4
:1001C00046E84ADF41E448DF40E046DFD1CF403730
:1001D00019F443E541DFCCCF483709F40DC1493765
:1001E00009F40AC1023179F0033169F0083359F09A
:1001F000083249F0003239F0063829F0013419F09C
:10020000083409F0F6C0403511F462DFF5C043341C
:10021000D1F429DF063809F4ECC038E438DF362F92
:1002200036DF352F34DF003409F44095342F2FDFCB
:10023000003421F0013411F010E223DF11E0222715
:10024000510F621FD9C04336C9F40DDF063821F0C3
:1002500030E41DDF362F03C0362F32D0326017DF77
:10026000352F15DF003409F44095342F10DF0034AA
:1002700021F0013411F010E204DFBEC0423521F557
:10028000063821F038E203DF362F03C0362F18D0AE
:100290003160FDDE352FFBDE0BDF432FDDDE063860
:1002A00009F466CF30E2F3DE362FF1DE352FEFDED4
:1002B000FFDE432FD1DE11E02227510F621F58CFFE
:1002C000330F330F330F0895413429F4CCDE642FFC
:1002D000CADE542F91C0443491F4C5DE063821F0B3
:1002E00030ECD5DE362F03C0362FEADF3660CFDEA6
:1002F000352FCDDE342FCBDE10E2C3DE7DC0443699
:1003000081F4063821F030EAC2DE362F03C0362FE2
:10031000D7DF3560BCDE352FBADECADE432F9CDE68
:1003200027CF4C3441F410E117BB063811F0C49AC2
:1003300063C0C49861C0453669F43CEAA8DE06385B
:1003400011F030E8A4DE34E0A2DE30E0A0DE10E3FD
:1003500098DE52C04C36A1F486DE3CEA98DE342F9B
:10036000063831F03670306E92DE30E090DE03C039
:10037000307E37608CDE30E08ADE10E382DE3CC007
:100380004337A1F4063809F434C0B2E005D0B1E037
:1003900003D0B0E001D0ECCE30E379DE30E077DEA0
:1003A0003B2F75DE85DE432F57DE08954D3659F419
:1003B0003CE46DDE362F6BDE352F69DE30E078DE13
:1003C0001FEF5FDE19C04A33A1F44DDEC42F4BDEB0
:1003D000D42F49DEE42F03D01FEF53DE0DC03C2F96
:1003E00056DE3D2F54DE3E2F52DE62DE432F34DEDA
:0E03F00008954FE331DEBCCE4DE02EDEB9CED7
:00000001FF
